:100000000C9485000C94AC0C0C94BF000C94BF00B5
:100010000C94BF000C94BF000C94BF000C942107FB
:100020000C94BF000C94BF000C94BF000C94BF0054
:100030000C94BF000C94BF000C94BF000C94BF0044
:100040000C94BF000C94BF000C94BF000C94BF0034
:100050000C94BF000C94BF000C94BF000C94BF0024
:100060000C94BF000C94BF000C94BF000C94BF0014
:100070000C94BF000C94BF000C94BF000C94BF0004
:100080000C94BF000C94BF000C94BF00740596053F
:10009000A705A705CC05D805160690059E06700590
:1000A0001A061D06220636064F066006F30564068C
:1000B0007F068206040309041003480065006E00F1
:1000C0006E0069006E0067002000420065006B0052
:1000D00065006C0012034B00650079006D00610043
:1000E0006E003600340012011001FF000008501DA0
:1000F000E96000010102000109021200010100C0D3
:100100003209040000000000000011241FBECFEFE0
:10011000D0E4DEBFCDBF04B603FE18C080917004EA
:1001200090917104A0917204B09173048F5E9E4B04
:10013000AD4ABE4D59F410927004109271041092A1
:10014000720410927304E0E0F0EE099513E0A0E071
:10015000B1E0E2EAF0E200E00BBF02C007900D92CE
:10016000A636B107D9F714E0A6E6B3E001C01D92A8
:10017000A037B107E1F70E94500A0C944F100C947D
:100180000000EF92FF920F931F93CF93DF93EC0148
:100190007A018B01B90120E030E040E050E016C068
:1001A000EA85FB85E40FF51F80819181A281B381EF
:1001B0004C5F5F4F8E159F05A007B10729F4FB0127
:1001C0003183208381E008C02F5F3F4F8C819D8168
:1001D0002817390728F380E0DF91CF911F910F9105
:1001E000FF90EF900895DC0120E030E01BC01696F0
:1001F000ED91FC911797A901440F551FE40FF51FCE
:100200000190F081E02D8181681751F41696ED91EF
:10021000FC911797E40FF51F0190F081E02D0AC0C3
:100220002F5F3F4F8D919C91119728173907F8F256
:10023000E0E0F0E0CF0108950E94F30020E0892B78
:1002400009F421E0822F0895FC0161830895F89458
:100250008FEE9EEBADEABEED809370049093710437
:10026000A0937204B09373042CE088E190E00FB681
:10027000F894A895809360000FBE20936000FFCF94
:1002800081E080937A0310927B0310927C0310929A
:100290007D0380910C0180937E0380919302809373
:1002A0007300E8E6F0E080818860808378940895A8
:1002B00088E10FB6F89480936000109260000FBE42
:1002C0008FEF81B980EC82B989E88AB980EF8BB968
:1002D0000E944001089581E080937A0310927B038D
:1002E00010927C0310927D0380910C0180937E0319
:1002F000089581E080937A0310927B0310927C032F
:1003000010927D0380910C0180937E03089581E01B
:1003100080937A0310927B038091660380937E031F
:10032000089580E090E0FC01E050FC4F808301964E
:1003300080349105C1F70895F999FECF8091680343
:100340009091690392BD81BDF89A80916803909164
:1003500069030196909369038093680380B590E0E8
:1003600008952091740330917503E0917203F09128
:100370007303E20FF31F80812F5F3F4F30937503AC
:100380002093740390E0089585B7806885BF85B792
:10039000806885BF08958BB190918F02892B8BB9AE
:1003A0008BB1909598239BB908958BB190918D0254
:1003B000892B8BB98AE18A95F1F78BB190959823B7
:1003C0009BB90895CF92DF92EF92FF920F931F9304
:1003D000CF93DF938BB190918F02892B8BB98BB127
:1003E000909598239BB9DD2400E010E0CC24C394C1
:1003F00020C089B190918E02892339F4F701E1542C
:10040000FC4FC082DD24D39406C0FE01E00FF11F33
:10041000E154FC4F10820E94D50121960894E11C02
:10042000F11CC830D10529F7085F1F4F00341105B2
:1004300021F07801C0E0D0E0DCCF8D2DDF91CF91AD
:100440001F910F91FF90EF90DF90CF9008959BB197
:1004500020919202822F809589238BB980EA9FE0B8
:100460000197F1F78BB1822B8BB908958BB19091E5
:100470009202892B8BB9E0EAFFE03197F1F78BB15B
:10048000909598239BB9089592B120919002822F64
:100490008095892382B982B1822B82B9089582B175
:1004A00090919002892B82B982B19095982392B94C
:1004B0000895282FE82FF0E0E158FC4F8081882331
:1004C00099F480919102662319F0922F982B03C022
:1004D000982F9095922380919002982B92B9E09159
:1004E0006C03F0916D03099508950F931F93CF93BB
:1004F000DF93182F062FC82FD0E0FE01E158FC4FE4
:100500008081882319F4812F0E945902FE01E1584D
:10051000FC4F00838081882321F4812F602F0E946B
:100520005902DF91CF911F910F910895CF93DF93DF
:10053000C0E0D0E0FE01E050FC4F8081FE01E154BC
:10054000FC4F60810E9459022196C034D10591F779
:10055000DF91CF910895DF93CF930F92CDB7DEB7A0
:100560008983898161E00E94590288EC90E020E94A
:1005700031E0F9013197F1F70197D9F7898160E00E
:100580000E9459020F90CF91DF910895DF93CF938E
:100590000F92CDB7DEB789838981EFEBF3E0E80FE7
:1005A000F11D80810F90CF91DF910895DF93CF935C
:1005B0000F92CDB7DEB789838981EFEBF3E0E80FC7
:1005C000F11D808191E089270F90CF91DF910895EF
:1005D000DF93CF930F92CDB7DEB78983898190E007
:1005E000803408F491E0892F0F90CF91DF91089526
:1005F000DF93CF930F92CDB7DEB7898389818034A3
:1006000040F50E94E201882321F1E981F0E0E15404
:10061000FC4F80818823E9F088EC90E020E931E00C
:10062000F9013197F1F70197D9F70E94E201882388
:1006300019F480E090E00EC0E981F0E0E154FC4F55
:10064000808190E0882309F491E081E09827892F48
:1006500001C080E00F90CF91DF910895DF93CF9399
:100660000F92CDB7DEB7898389818034E0F40E9490
:10067000E201E981F0E0E154FC4F8081882399F4A4
:1006800088EC90E020E931E0F9013197F1F701972A
:10069000D9F70E94E201E981F0E0E154FC4FE081EA
:1006A00081E0E82701C0E0E08E2F0F90CF91DF912D
:1006B0000895A0914004B09141041C96ED91FC91E5
:1006C0001D97808184B91C96ED91FC911D978181C5
:1006D00085B91C96ED91FC911D97828187B91C9676
:1006E000ED91FC911D97838188B908950E94890E30
:1006F00008950E94890E08950F931F93CF93DF935F
:100700008C01C0E0D0E00AC0CE01880F991FE80F2D
:10071000F91F808191810E94890E2196D8018C91C8
:1007200090E01396ED91FC911497C817D90764F3E4
:10073000CF010E94890EC8010E94890EDF91CF91DE
:100740001F910F9108950F931F93CF93DF938C0107
:10075000C0E0D0E00AC0CE01880F991FE80FF91F52
:10076000808191810E947C032196D8018D919C917A
:1007700011971696ED91FC911797C817D90758F362
:10078000CF010E94890EC0E0D0E00AC0CE01880FE0
:10079000991FE80FF91F808191810E94890E21968F
:1007A000F801828193810084F185E02DC817D90773
:1007B00068F3CF010E94890ED8011A968D919C9101
:1007C0001B970E94890EC8010E94890EDF91CF916C
:1007D0001F910F910895FC018181882321F08130C0
:1007E00031F180E008958681978190937103809321
:1007F00070038281938190937703809376031092A4
:100800006F0310926E038091720390917303892B92
:1008100061F4609170037091710381E090E00E9437
:10082000C00D80937203909373038FEF0895E0914E
:100830004004F09141048485958590935104809300
:10084000500484E0089581E090E064E070E00E944C
:10085000C00D089581E090E065E070E00E94C00D59
:10086000FC0188E0808311828FEF8283838314826E
:100870008E2F0895FF920F931F9381E090E065E023
:1008800070E00E94C00DF92E082F192F81E090E032
:1008900062E070E00E94C00DF80183839483809130
:1008A0000801818380E48283802F9F2D1F910F9107
:1008B000FF900895FF920F931F9381E090E06EE008
:1008C00070E00E94C00DF92E082F192F81E090E0F2
:1008D00062E070E00E94C00DF80186839783118664
:1008E00010861386128681E090E064E070E00E943A
:1008F000C00DF801848795871182108213821282BD
:1009000015821482802F9F2D1F910F91FF900895C3
:10091000A0914004B09141041C96ED91FC911D976B
:1009200084B180831C96ED91FC911D9785B18183E4
:100930001C96ED91FC911D9787B182831C96ED91D9
:10094000FC911D9788B183831C96ED91FC911D97B6
:1009500082E090E060810E944110E0914004F091BB
:1009600041040484F585E02D83E090E061810E94DC
:100970004110E0914004F09141040484F585E02D9C
:1009800084E090E062810E944110E0914004F09187
:1009900041040484F585E02D85E090E063810E94A8
:1009A000411008954F925F926F927F928F929F9223
:1009B000AF92BF92CF92DF92EF92FF921F93CF93AD
:1009C000DF936C01EE24FF2470E9472E71E0572E6F
:1009D00060EA662E6FE0762E49C0F601EE0DFF1D2F
:1009E000808190E0FC01EE0FFF1FE80FF91FE35F2D
:1009F000FE4F828180809180C0E0D0E0A82EBB2491
:100A00002FC0F401EC0FFD1F8081282F30E0207CE7
:100A100030702038310519F48F7361E005C020343F
:100A2000310541F48F7360E00E945902C3010197C0
:100A3000F1F715C0203C310591F4182F1F738091F8
:100A40007903181739F488EC90E0F2013197F1F747
:100A50000197D9F7812F0E94AB0210937903219659
:100A6000CA15DB0574F20894E11CF11CF601019033
:100A70000020E9F73197EC19FD09EE16FF0608F49E
:100A8000ACCFDF91CF911F91FF90EF90DF90CF908F
:100A9000BF90AF909F908F907F906F905F904F909E
:100AA0000895CF93DF939C01EB018981882329F07E
:100AB00047E250E0A8E2B0E004C044E250E0A5E222
:100AC000B0E08881E82FF0E0E431F10508F036C1AC
:100AD000EA5BFF4FEE0FFF1F0590F491E02D0994A4
:100AE0008B818093FF032AC16A81262F90E002C088
:100AF00026959F5F20FFFCCF8B81282330E002C02A
:100B0000220F331F9A95E2F78C91609586238C9380
:100B10008C91822B8C93DA018C919A81892B3AC02B
:100B2000FA0180819A81892B80833CC02C913A8183
:100B30002323FA018081832B80839C918A81809575
:100B400098239C938C912327282B2C93F7C06A81A0
:100B50002C91823011F03FEF01C031E02623862F27
:100B600090E003C0869526959F5F80FFFBCF230F03
:100B7000282330E002C0220F331F9A95E2F7FA01D2
:100B80008081862B80839C918A81809598239C9379
:100B90008C91822B8C93D2C0FA0190818A818095AE
:100BA000982390839C918A81809598239C93C6C0BA
:100BB0009B8180E02A8130E0822B932B9C0144278B
:100BC00037FD4095542F60EA7FE007C0CB010197C5
:100BD000F1F721503040404050402115310541058A
:100BE0005105A1F7ABC0D9011A96ED91FC911B9765
:100BF0009B8180E02A8130E0822B932B880F991F04
:100C0000880F991FE80FF91F80819181A281B3811C
:100C100020EA3FE006C0F9013197F1F70197A109F9
:100C2000B1090097A105B105B1F788C08B810E9479
:100C3000DB0684C08B8161E002C08B8160E00E9492
:100C400059027CC0D9011896ED91FC9119979B81AE
:100C500080E02A8130E0822B932B880F991FE80FC8
:100C6000F91F808191810E94D20468C0F8948FEEB0
:100C70009EEBADEABEED8093700490937104A09357
:100C80007204B09373042CE088E190E00FB6F894FE
:100C9000A895809360000FBE20936000FFCFAA81CB
:100CA000B0E0A050BC4F9C91EB81F0E0E050FC4FD5
:100CB00080818C93EB81F0E0E050FC4F90833EC04C
:100CC0008B810E94AB023AC06B81662349F487E2B4
:100CD00092E090936B0380936A0384E492E00AC0ED
:100CE000613061F586E392E090936B0380936A0331
:100CF0008FE492E090936D0380936C031FC00E9479
:100D000088041CC0A0914004B09141041C96ED9150
:100D1000FC911D97808184B91C96ED91FC911D97E3
:100D2000818185B91C96ED91FC911D97828187B9CF
:100D30001C96ED91FC911D97838188B9DF91CF912D
:100D400008950F931F93CF93DF93EC0100E010E021
:100D500021C0C801880F991FEB81FC81E80FF91FA2
:100D60000190F081E02D8481882359F0803421F4B2
:100D70008A81803469F405C0803651F48A818036D6
:100D800039F48091400490914104BF010E945105C3
:100D90000F5F1F4F888190E008171907D4F28A81EE
:100DA000803411F080E401C080E68A83DF91CF9126
:100DB0001F910F9108951F93CF93DF93182FC0E0D9
:100DC000D0E012C00680F781E02DCE01880F991F78
:100DD000E80FF91F0190F081E02D8181181719F4B7
:100DE000CF010E94A1062196E0914004F0914104B8
:100DF00080819181C817D90728F3DF91CF911F9186
:100E00000895823071F0833018F48130C9F405C040
:100E1000833051F08430A1F410C0862F0E94DB068D
:100E20000895862F61E002C0862F60E00E9475025F
:100E300080EA9FE00197F1F70895862F0E94AB02A8
:100E400008951F920F920FB60F920BB60F921124B6
:100E50002F933F934F935F936F937F938F939F93C2
:100E6000AF93BF93EF93FF9389B19091930289233E
:100E700009F046C089B190919402892339F090918C
:100E80007B0380917A03892B80937B0380917A0383
:100E9000880F80937A0390917A0380917E0398174C
:100EA00079F590917E0380910C012091660398174B
:100EB00061F480917B0380937C0381E080937A03CB
:100EC00010927B0320937E031BC080917E038217C8
:100ED000B9F480917B0380937D0380917C036091C2
:100EE0007D030E94010781E080937A0310927B03C7
:100EF00010927C0310927D0380910C0180937E03FD
:100F0000FF91EF91BF91AF919F918F917F916F91E1
:100F10005F914F913F912F910F900BBE0F900FBE9D
:100F20000F901F9018958F929F92AF92BF92CF9281
:100F3000DF92EF92FF920F931F93CF93DF938C0179
:100F40005B01CC24DD2460EA862E6FE0962E48C03B
:100F5000D8011696ED91FC9117977601EE0CFF1CC7
:100F6000EE0DFF1D0190F081E02D9181809108012F
:100F7000981799F5C0E0D0E021C0D8011696ED9100
:100F8000FC911797EE0DFF1D0190F081E02DCE0131
:100F9000880F991F0380F481E02DE80FF91F60810D
:100FA0007181C8010E945105A114B10431F0C5013D
:100FB000F4013197F1F70197D9F72196D8011696E8
:100FC000ED91FC911797EE0DFF1D0190F081E02D42
:100FD000808190E0C817D90784F20894C11CD11C05
:100FE000F80180819181C816D90608F4B1CFDF914C
:100FF000CF911F910F91FF90EF90DF90CF90BF9016
:10100000AF909F908F900895F8940E94820B519A10
:1010100088E893E120E931E0F9013197F1F7019790
:10102000D9F751987894109273031092720308952F
:10103000EF92FF920F931F937C018B01CB010E94D3
:10104000E50FF7018083C8010E94E50FF701818356
:10105000C8010E94E50FF7018283C8010E94E50FD5
:10106000F70183831F910F91FF90EF9008950F93E5
:101070001F93CF93DF93EC018B01CB010E94E50F0F
:101080008883198287FF02C081E089838881982F35
:1010900090769C838F718883C8010E94E50F8A83B4
:1010A000C8010E94E50F8B83DF91CF911F910F91B3
:1010B0000895EF92FF920F931F938C01F62EE72E67
:1010C000DC016C9170E06F5F7F4F660F771F1396A6
:1010D0008D919C9114970E94E10EF8019483838373
:1010E000E081F0E0EE0FFF1FE80FF91FF082E182D0
:1010F000D8018C918F5F8C938F2D9E2D1F910F9116
:10110000FF90EF900895CF92DF92EF92FF920F93AE
:101110001F93CF93DF936C018B01CB010E94E50FEE
:10112000C0E0D0E0E82EFF240AC00E942A04BC01DF
:10113000C6010E945908B8010E9437082196CE15B1
:10114000DF059CF3DF91CF911F910F91FF90EF90FE
:10115000DF90CF900895EF92FF920F931F938C0131
:10116000F62EE72EDC0116968D919C9117976D91C6
:101170007C916F5F7F4F660F771F0E94E10EF80131
:10118000978386830680F781E02DD8018D919C910D
:101190001197880F991FE80FF91FF082E1828D9156
:1011A0009C911197019611969C938E938F2D9E2D55
:1011B0001F910F91FF90EF900895CF92DF92EF92E1
:1011C000FF920F931F938C016A017B01DC011A9639
:1011D0008D919C911B9714966D917C9115976F5FE3
:1011E0007F4F660F771F660F771F0E94E10EF80191
:1011F000938782870284F385E02DD80114968D9120
:101200009C911597880F991F880F991FE80FF91F58
:10121000C082D182E282F38214968D919C911597BF
:10122000019615969C938E93149714962D913C914C
:10123000159721503040C9011F910F91FF90EF90F9
:10124000DF90CF900895AF92BF92CF92DF92EF924E
:10125000FF920F931F937C01B62EA72EFC01808571
:101260009185628173816F5F7F4F660F771F0E9448
:10127000E10EF70191878087C084D18402811381B8
:10128000EB2DFA2DDF010D900020E9F7CD018E1B2B
:101290009F0B61E070E00E94C00D000F111F0C0D4C
:1012A0001D1DF80180839183F7012085318582819E
:1012B0009381EB2DFA2DDF010D900020E9F71197B6
:1012C000AE1BBF0B880F991F280F391FF9018081B2
:1012D00091816B2D7A2DAD010E94D60FF70182818D
:1012E0009381019693838283228133812150304000
:1012F000C9011F910F91FF90EF90DF90CF90BF90A9
:10130000AF9008952F923F924F925F926F927F928B
:101310008F929F92AF92BF92CF92DF92EF92FF9205
:101320000F931F93DF93CF93CDB7DEB7C050D0415B
:101330000FB6F894DEBF0FBECDBF1C012B01CB0151
:101340000E94E50F982F80910501981741F4C20182
:101350000E94E50F982F80910601981739F0892F88
:1013600090E0B2010E94271080E080C0F1018485E6
:101370009585B2010E9418086FC080910901181765
:1013800001F500E010E009C0E1E0F0E0EC0FFD1F26
:10139000E00FF11F80830F5F1F4FC2010E94E50F16
:1013A000882391F781E090E08C0F9D1F080F191F93
:1013B000F8011082C101BE016F5F7F4F0E942309B7
:1013C0004BC080910A011817E1F5C2010E94E50F98
:1013D0003C01C2010E94E50F7C01C2010E94E50FA1
:1013E0005C01C2010E94E50F0027F7FC0095102F59
:1013F000102F0F2DFE2CEE24CC24B7FCC094DC2C37
:101400006501BB24AA24EA28FB280C291D2988246D
:1014100077FC8094982CE628F72808291929AA2710
:1014200097FDA095BA2FB82FAA2799278827E82AD1
:10143000F92A0A2B1B2BC101B801A7010E94DD0864
:101440000BC00E943A04BC01C1010E94AB08FC0120
:101450001183B2010E948308C2010E94E50F182F78
:1014600080910701181709F088CF81E0C050D04F54
:101470000FB6F894DEBF0FBECDBFCF91DF911F91A5
:101480000F91FF90EF90DF90CF90BF90AF909F9023
:101490008F907F906F905F904F903F902F90089526
:1014A000EF92FF920F931F93CF93DF930E94580107
:1014B00080E090E0FC01E050FC4F80830196803496
:1014C0009105C1F780910B018093FF0386E392E0C1
:1014D00090936B0380936A038FE492E090936D0383
:1014E00080936C030E945A048093400490934104BB
:1014F00065E972E00E948209809140049091410464
:1015000060E070E00E949307E0916A03F0916B0342
:1015100009950E940408FF24F394EE24E3940E94AA
:10152000890B80916703882319F08130C1F70EC0C1
:101530008091FF030E94F802882329F0E09267035C
:10154000FF24F394ECCF0E949602E9CF8091FF0331
:101550000E942E03882319F400E010E023C0FF202E
:1015600021F08091FF030E94AB0210926703D7CF56
:101570000680F781E02DC801880F991FE80FF91F39
:10158000C081D18189810E94F802882349F0CE016F
:101590000E94A10689810E942E038823D9F3FF248B
:1015A0000F5F1F4FE0914004F091410480819181D1
:1015B00008171907E8F2B3CF0F931F930E945A043C
:1015C000182F092F109275031092740363EA72E0CA
:1015D0000E948209882341F060917603709177031D
:1015E000812F902F0E949307812F902F0E94A30399
:1015F0001F910F9108950F931F93CF93DF938C0149
:10160000C0917203D091730340E050E070E016C0C7
:10161000E0916E03F0916F03EC0FFD1FD801A40F52
:10162000B51F8C9180834F5F5F4F80916E039091C7
:101630006F03019690936F0380936E0320916E0366
:1016400030916F03809170039091710328173907CF
:1016500018F446175707E4F220916E0330916F0398
:1016600080917003909171032817390710F480E07E
:101670000DC00E94DC0A80917203909173030E9456
:10168000890E109273031092720381E0DF91CF9163
:101690001F910F910895CF92DF92EF92FF920F93D7
:1016A0001F93CF93DF938C017B016A01C0E0D0E0F0
:1016B00017C0D8011896ED91FC911997CE01880FAB
:1016C000991FE80FF91F80819181B7010E94CD0F0A
:1016D000009729F4F601D183C08381E00AC02196E6
:1016E000D80112968D919C911397C817D90708F3CA
:1016F00080E0DF91CF911F910F91FF90EF90DF90ED
:10170000CF900895E9E6F0E0808182608083E89AD6
:1017100008951F93CF93DF9360915204635067FD48
:10172000A6C080914F04CCE0D0E0C81BD109CA5AB2
:10173000DB4F80914E048D3209F086C0683009F08D
:1017400094C083EC809342048AE580935E031092F8
:1017500078039881892F807641F0CE010E94EB03B7
:10176000282F8F3F09F45FC065C02A8110924B0477
:101770008981882349F49F7119F481E080934B0497
:1017800010924C0422E048C0853019F42093530491
:1017900042C0863089F58B81813019F486EE90E065
:1017A00020C0823019F488EF90E01BC08330F9F438
:1017B0008A81882341F484EB90E0909351048093D4
:1017C000500424E015C0813041F488EB90E0909300
:1017D0005104809350042CE10BC0823041F484ED1D
:1017E00090E0909351048093500422E101C020E0E6
:1017F00080E4809378031EC0883021F421E085E5E1
:1018000094E00CC0893019F42093550404C08A3048
:1018100011F421E001C020E08BE494E090935104A6
:101820008093500407C0888187FD2E8180E88093D3
:10183000780306C08F81882319F48E81821708F0FF
:10184000822F80935F0311C08091780387FF0DC0C2
:10185000CE010E94FB0A8F3F21F48EE180935E034C
:1018600004C0882311F010925F03109252048091FB
:101870005E0384FF4AC080915F038F3F09F445C037
:10188000182F893008F018E0811B80935F03809146
:10189000420498E8892780934204112341F1209162
:1018A0005004309151048091780386FF0DC0A3E469
:1018B000B4E080E090E0F901E80FF91FE491ED93C6
:1018C00001961817C1F708C0912FD901E3E4F4E09D
:1018D0008D9181939150E1F71150812F90E01F5F1E
:1018E0000196820F931F909351048093500483E4D8
:1018F00094E0612F0E94A80C612F6C5F6C3019F08E
:101900008FEF80935F0360935E0394E189B18670EB
:1019100031F49150D9F71092530410924D04DF9195
:10192000CF911F910895A82FB92F80E090E041E05A
:1019300050EA609530E009C02D91822797958795F0
:1019400010F084279527305EC8F36F5FA8F30895E1
:10195000EADF8D939D930895CF93CFB7CF93DF9315
:10196000C395499BE9F7499B0BC0499B09C0499B1B
:1019700007C0499B05C0499B03C0499B01C089C062
:101980006F93C0914F04DD27CA5ADB4F2F9365E553
:10199000499B03C02F916F91E6CF0F931F934F93F5
:1019A00020E040E15F9309B1067001FB27F93F9306
:1019B00050E03BE039C0167040642F77012F5F5F25
:1019C0001EC0406819B116702F7752501FC0406476
:1019D00009B12F770670D1F15F5F00C023C040626C
:1019E00019B12F77167091F15F5F00C025C00670A6
:1019F0001027515012F45D5F0000115027952C3FC5
:101A000019B1C8F616700127015027952C3FC8F66A
:101A10004227499309B1067010274F73115027953B
:101A20002C3FA8F64695469519B1167079F0012716
:101A3000015027952C3F98F66B5A60F3315009B14D
:101A4000B0F600C011E01CBB002717C03B50319519
:101A5000C31BD04011E01CBB0881033CF9F00B34E0
:101A6000E9F020914D041981110F1213EDCF0936C1
:101A700051F10D3211F0013E39F7009354043F91BA
:101A80005F914F911F910F912F916F91CCB3C0FD3A
:101A900067CFDF91CF91CFBFCF911895209154049C
:101AA000222369F310915204112339F534303AF1AD
:101AB0003093520420934E0410914F043BE0311BAD
:101AC00030934F041CC0009152040130B4F40AE575
:101AD00030915E0334FD14C000935E03C2E4D4E091
:101AE00013C0052710E000C000000BB91AC005277D
:101AF00010E0221F1DC010E021C04AE502C032EDF7
:101B0000432FC4E1D0E032E01AB11660599A0BB10C
:101B10001AB956E020E865E320FF05270BB92795A1
:101B200017951C3FF0F66695B8F7B1F720FF05272B
:101B30000BB9279517951C3FD0F62795179517FFDA
:101B4000052700001C3F0BB9B0F629913A9519F70B
:101B5000097F10915304110FC651D0400BB911F0F9
:101B600010934D0411E01CBB02601AB1197F402F85
:101B7000497F54E05A95F1F70BB91AB94BB97FCFA9
:101B80000F931F93CF93DF93689F8001699F100D80
:101B9000789F100D1124C8010E94DC0DEC01009704
:101BA00029F060E070E0A8010E94C60FCE01DF912D
:101BB000CF911F910F910895CF93DF93BC01823095
:101BC000910510F462E070E0A0916E04B0916F0492
:101BD000ED01E0E0F0E040E050E021C08881998133
:101BE0008617970769F48A819B81309719F0938350
:101BF000828304C090936F0480936E04FE0134C00E
:101C00006817790738F44115510519F084179507BD
:101C100008F4AC01FE018A819B819C01E9012097B7
:101C2000E9F641155105A9F1CA01861B970B0497E6
:101C300008F4BA01E0E0F0E02AC08D919C91119780
:101C400084179507F9F46417750781F412968D913E
:101C50009C911397309719F09383828304C09093DB
:101C60006F0480936E04FD0132964FC0CA01861B3B
:101C7000970BFD01E80FF91F6193719302978D9304
:101C80009C9343C0FD01828193819C01D9011097EF
:101C9000A1F680916C0490916D04892B41F48091A0
:101CA00062039091630390936D0480936C04409160
:101CB0006403509165034115510541F44DB75EB77A
:101CC0008091600390916103481B590B20916C0433
:101CD00030916D0424173507B0F4CA01821B930BB1
:101CE0008617970780F0AB014E5F5F4F841795070B
:101CF00050F0420F531F50936D0440936C04F90150
:101D00006193719302C0E0E0F0E0CF01DF91CF91E9
:101D10000895CF93DF93009709F450C0EC01229708
:101D20001B821A82A0916E04B0916F04109709F182
:101D300040E050E0AC17BD0708F1BB83AA83FE0169
:101D400021913191E20FF31FAE17BF0779F48D9106
:101D50009C911197280F391F2E5F3F4F398328839D
:101D600012968D919C9113979B838A8341155105FF
:101D700071F4D0936F04C0936E0420C012968D91BD
:101D80009C911397AD01009711F0DC01D3CFFA01BC
:101D9000D383C28321913191E20FF31FCE17DF0766
:101DA00069F488819981280F391F2E5F3F4FFA010E
:101DB000318320838A819B8193838283DF91CF91BA
:101DC00008958F929F92AF92BF92CF92DF92EF923F
:101DD000FF920F931F93CF93DF938C01009729F409
:101DE000CB010E94DC0D8C01BAC09EEFE92E9FEF63
:101DF000F92EE00EF11E5801A60EB71EAE14BF0458
:101E000008F4ABC08EEF882E8FEF982E8A0C9B1CA7
:101E1000E7014881598146175707B8F04530510509
:101E200008F49DC0CA0104978617970708F497C065
:101E300042505040461B570BF40151834083798335
:101E40006883C5010E94890E8AC06B01C41AD50A35
:101E5000E0916E04F0916F04A0E0B0E0C0E0D0E04B
:101E600042C0E815F905A1F5208131812C153D0509
:101E700078F1C90102968C159D05A8F04E5F5F4F61
:101E8000420F531FE7015983488322813381109702
:101E900029F013963C932E93129761C030936F04F0
:101EA00020936E045CC0225030402C193D093183D0
:101EB0002083109729F01396FC93EE93129704C099
:101EC000F0936F04E0936E04F7017183608347C061
:101ED00080819181C817D90708F4EC01DF01828164
:101EE00093819C01F901309709F0BBCF400F511F3E
:101EF00080916C0490916D0484179507E9F4C617DE
:101F0000D707D0F420916403309165032115310582
:101F100041F42DB73EB78091600390916103281B77
:101F2000390BA216B306C8F4B0926D04A0926C04EB
:101F3000E7017983688313C0CB010E94DC0DEC01BB
:101F4000009759F0F70140815181B8010E94BD0FFF
:101F5000C8010E94890E8E0102C000E010E0C80195
:101F6000DF91CF911F910F91FF90EF90DF90CF9075
:101F7000BF90AF909F908F900895FB01DC0102C04D
:101F800001900D9241505040D8F70895DC0101C0F6
:101F90006D9341505040E0F70895FB01DC018D91B5
:101FA000019080190110D9F3990B0895FB01DC0110
:101FB0004150504048F001900D920020C9F701C0F7
:101FC0001D9241505040E0F70895CF93DF93EC010C
:101FD0004B8140FF1AC046FF0AC04F7B4B838E8166
:101FE0009F8101969F838E838A81282F2BC042FF79
:101FF00013C0E881F9818081282F332727FD309590
:102000002115310529F440624B832FEF3FEF1BC0B0
:102010003196F983E88311C0EA85FB85CE010995E5
:102020009C0197FF0AC09B812F5F3F4F11F080E218
:1020300001C080E1892B8B83E8CF8E819F8101963F
:102040009F838E8330E0C901DF91CF9108959C0179
:10205000FB01838180FF11C086FD0FC09FEF2F3FE2
:10206000390759F0228380648F7D8383868197812D
:1020700001979783868330E002C02FEF3FEFC901BD
:102080000895262FF999FECF1FBA92BD81BD20BDBC
:102090000FB6F894FA9AF99A0FBE01960895F8943B
:0220A000FFCF70
:1020A20000406040601CCFFFFEFDFC0F1068030083
:1020B200680300680300680300680300680300689F
:1020C20003006803006803006803006803006803F4
:1020D20000680300B102016803006803006803009E
:1020E200680300680300680300680300680300686F
:1020F20003006803006803006803006803006803C4
:1021020000680300680300680300680300B202016C
:10211200B30203B60203B90203BC0203BF0203C245
:102122000203C50203C80203CB0203CE0201CF029F
:1021320001D00201D10201D20201D30201D4020173
:10214200D50201D60201D70201D80201D90201DA71
:102152000201DB0201DC0201DD0201DE0201DF021B
:1021620001E00203E30201E40203E70203EA0201DF
:10217200EB0203EE0203F10203F40203F70203FA95
:102182000203FD020300030303030306030309031F
:10219200030C03030F0303120303150303180303C2
:1021A2001B03031E03032103032403032703032A40
:1021B20003032D03033003033303033603033903FD
:1021C200033C03013D030340030168030041030193
:1021D200420301430301440301450301460301474E
:1021E20003014803014903014A03014B03014C0364
:1021F200014D03014E03014F03015003015103013D
:1022020052030153030154030155030156030157BD
:1022120003015803015903015A03015B03016803D7
:10222200006803006803005C03015D0301081001FC
:102232004080804020000000010000000000009C5F
:1022420001000000000001000000000000B10100D8
:1022520000C8E7B9C779B9DF79B9C179B9D979B90C
:10226200C279B9DA79B9C379B9DB79B9C479CEC59A
:10227200FDDDE5FEDCC7DFC1D9C2DAC3DBC4EDD6C2
:10228200B9FD79EEB9E579B9FE79F5B9D179B9E354
:1022920079B9E279B9D279B9F179B9EA79B9D37967
:1022A200B9EB79B9CC79B9D479B9EC79B9D579B92D
:1022B200E479B9FC79B9F479B9CD79B9F779B9CAC0
:1022C20079B9E979B9F279B9F379B9FB79B9C97907
:1022D200B9FA79B9CB79B9E179B9ED79C6B9D679D3
:1022E200F6CFD1E3E2D2F1EAD3EBCCD4ECD5E4FCE5
:1022F200F4CDF7CAE9F2F3FBC9FACBE1C8C05AFF41
:062302002000740400003D
:00000001FF
